:020000040000FA
:1000000024EF14F0120012000EEF00F012000100B5
:10001000CA2800000001000074000000DACFE4FFED
:10002000E2CFDAFFE9CFE4FFEACFE4FFF6CFE4FF67
:10003000F7CFE4FFF5CFE4FFF3CFE4FFF4CFE4FF25
:10004000FACFE4FF00EE00F0140EE80403E3EECF75
:10005000E4FFFBD700EE14F0070EE80403E3EECF55
:10006000E4FFFBD7E6529D50200B30E09E50200B62
:100070002DE097EC13F00F010F6FABA407D0AB9EF0
:100080001E810D2B000E0E23AB8E01D01E91ABA254
:1000900007D0AB981E83AB880B2B000E0C2301D02E
:1000A0001E93ACA2FED70F0104CFE9FF05CFEAFFF4
:1000B000042B000E05230FCFEFFFB00E045D000EE2
:1000C000055904E3600E046F000E056FE55200EE63
:1000D0001AF0070EE80403E3E5CFEDFFFBD700EECF
:1000E00013F0140EE80403E3E5CFEDFFFBD7E5CFF3
:1000F000FAFFE5CFF4FFE5CFF3FFE5CFF5FFE5CF5E
:10010000F7FFE5CFF6FFE5CFEAFFE5CFE9FFE5CF63
:10011000DAFF1100D9CFE6FFE1CFD9FFE652FE0E9C
:10012000DB50DF6EDF0601E0FDD7E552E552E7CF99
:10013000D9FF1200D9CFE6FFE1CFD9FFE652D9505F
:10014000FD0FE96EFF0EDA20EA6EEE50ED1001E1D0
:1001500014D0050EDF6EA40EE66EDCDFE552DF067E
:10016000FAE1FD0EDB06DBCF14F0FE0E01E2DB064A
:10017000DBCF15F014501510ECE1E552E552E7CF56
:10018000D9FF12008168010E936E0F01396B070EC3
:10019000806E386B388138830F0E926E806A826869
:1001A0003A6BBF0E946E948E949C606A1200200E7F
:1001B000E66EE66A740EE66ED5EC12F0E552E55294
:1001C000E5529F8AD08E9D9AF28CF29E1200D9CF72
:1001D000E6FFE1CFD9FF020EE126DE6ADD6AFD0E01
:1001E000DBCFF6FFFE0EDBCFF7FF0800F55015E082
:1001F000FD0EDBCFF6FFFE0EDBCFF7FF0800F5505C
:10020000E66E55D8E552DF2A010E01E3DB2AFD0E2A
:10021000DB2AFE0E01E3DB2AE2D7DECF14F0DDCFCE
:1002200015F014C0F3FF15C0F4FF020EE15C03E209
:1002300000D0E16AE552E16EE552E7CFD9FF120046
:10024000D9CFE6FFE1CFD9FF020EE126DE6ADD6AF3
:10025000FD0EDBCFE9FFFE0EDBCFEAFFEF5014E02F
:10026000FD0EDBCFE9FFFE0EDBCFEAFFEF50E66EBF
:100270001ED8E552DF2A010E01E3DB2AFD0EDB2A40
:10028000FE0E01E3DB2AE4D7DECF14F0DDCF15F05C
:1002900014C0F3FF15C0F4FF020EE15C03E200D0CE
:1002A000E16AE552E16EE552E7CFD9FF1200D9CFFE
:1002B000E6FFE1CFD9FFACA2FED7FE0EDBCFE6FF13
:1002C000EBEC13F0E552E552E7CFD9FF12000D0E2B
:1002D000E66EEDDFE5520A0EE66EE9DFE55212004A
:1002E000D9CFE6FFE1CFD9FFE6520F010451021941
:1002F00002E10551031901E1F8D702CFE9FF03CF6D
:10030000EAFF022B000E0323EFCFDFFFB00E025DEA
:10031000000E035904E3600E026F000E036FDF50FE
:1003200000D0E552E552E7CFD9FF12000F01600E71
:10033000046F000E056F04CF02FF05CF03FF216B92
:10034000226B0F6B076B1200D9CFE6FFE1CFD9FF0D
:10035000FF0EE76EFD0EDBCF14F0FE0EDBCF15F0C7
:10036000E7501416156A1450A96EFD0EDBCF14F079
:10037000FE0EDBCF15F015C014F0156A030E141431
:10038000AA6EA69EA69CA680E80EE66E030EE66EFA
:10039000E66AE66AB4D9E552E552E552E552A8505C
:1003A00000D0E552E7CFD9FF1200D9CFE6FFE1CF69
:1003B000D9FF020EE1260F011DAF11D0E76EFD0E31
:1003C000DBCF14F0FE0EDBCF15F0E7501426000E45
:1003D0001522FD0E14C0DBFFFE0E15C0DBFFFD0E67
:1003E000DBCF14F0FE0EDBCF15F015C014F0156A4C
:1003F000030E1414AA6EFF0EE76EFD0EDBCF14F091
:10040000FE0EDBCF15F0E7501416156A1450A96ED6
:10041000FC0EDB50A86EA69EA684A69CF2AE04D06D
:10042000F29E010EDE6EDD6A550EA76EAA0EA76E55
:10043000A682A1A8FED7A198A694D9CFE9FFDACFCA
:10044000EAFF010EEE1801E1ED5001E1F28E020E1D
:10045000E15C02E2E16AE552E16EE552E7CFD9FFE5
:100460001200D9CFE6FFE1CFD9FFFB0EDBCFE9FFCA
:10047000FC0EDBCFEAFFEF5022E0FB0EDBCFE9FF03
:10048000DB2AFC0EDBCFEAFF01E3DB2AEF50E66E4E
:10049000D950FD0FE96EFF0EDA20EA6EEECF14F0B0
:1004A000EDCF15F0020EEE26000EEF2214C0E6FF8F
:1004B00015C0E6FF7ADFE552E552E552D6D7E552A0
:1004C000E7CFD9FF1200D9CFE6FFE1CFD9FF040E65
:1004D000E1260F011DAF17D0FD0EDBCF14F0FE0E8D
:1004E000DBCF15F0040ED89014361536E804FBE186
:1004F000000E1426020E1522FD0E14C0DBFFFE0EA8
:1005000015C0DBFF12D0FD0EDBCF14F0FE0EDBCFEB
:1005100015F0050ED89014361536E804FBE1FD0EF3
:1005200014C0DBFFFE0E15C0DBFF020EDB6A030EFC
:10053000DB6AD950FD0FE96EFF0EDA20EA6EFF0E7E
:10054000D880EE54030EED5401E228D0FD0EDBCF2F
:10055000E6FFFE0EDBCFE6FFF7DEE552E552DE6E8C
:10056000DD6AD9CFE9FFDACFEAFFEE50ED1001E105
:1005700015D0DFCFE6FF9BDEE552FD0EDB2AFE0E37
:1005800001E3DB2A020EDB2A030E01E3DB2AD9CFCB
:10059000E9FFDACFEAFFEE50ED10CBE1E80EE66EB0
:1005A000030EE66EE66AE66AAAD8E552E552E5521F
:1005B000E552040EE15C02E2E16AE552E16EE552C9
:1005C000E7CFD9FF1200D9CFE6FFE1CFD9FF040E64
:1005D000E1260F015E0E006F010E016F00CFE6FFF6
:1005E00001CFE6FFFD0EDBCFE6FFFE0EDBCFE6FF21
:1005F00095EC0FF0E552E552E552E55200CFE6FFEB
:1006000001CFE6FF20EC12F0E552E552F3CFDEFF1A
:10061000F4CFDDFFD9CFE9FFDACFEAFF020EEECF4C
:10062000DBFF030EEDCFDBFF020EDBCF14F0030E7A
:10063000DBCF15F0040E145C000E15580AE2300EE4
:10064000E66E35DEE552020EDB2A030E01E3DB2AFD
:10065000EBD700CFE6FF01CFE6FFF2DDE552E55232
:10066000F3CFDEFFF4CFDDFF040EE15C02E2E16ACE
:10067000E552E16EE552E7CFD9FF1200D9CFE6FF90
:10068000E1CFD9FF020EE126010EDB6AFE0EDB5040
:10069000F00BE8380F0B300FDF6EDF50390803E244
:1006A000070EDF24DF6EFE0EDB500F0B300FE76E00
:1006B000010EE7CFDBFFDB5039080AE2070E146EAC
:1006C000010EDBCFE7FF1450E726010EE7CFDBFF7B
:1006D000DFCFE6FFECDDE552010EDBCFE6FFE7DD25
:1006E000E552680EE66EE3DDE552020EE15C02E2E1
:1006F000E16AE552E16EE552E7CFD9FF1200D9CFAA
:10070000E6FFE1CFD9FFFB0EDBCF05F0FC0EDBCF20
:1007100006F0FD0EDBCF07F0FE0EDBCF08F008344D
:10072000000E081809E6D880000E0554000E065485
:10073000000E0754000E08540CE2D950FB0FE96E6E
:10074000FF0EDA20EA6EEE06000EEE5AEE5AEE5A70
:10075000DAD7E552E7CFD9FF1200C280C19EC08E22
:10076000C08AC088C096C082C094C090C196C1940F
:10077000C192C1901200D9CFE6FFE1CFD9FF040E9C
:10078000E126FD0EDBCF14F0FE0EDBCF15F0D89086
:1007900014361536D89014361536010E1424C26E50
:1007A0000A0EE66E40EC14F0E55262EC14F05DECDB
:1007B00014F0000901E0FBD74BEC14F0F3CFDEFF9F
:1007C000F4CFDDFFDECF14F0DDCF15F014C0F3FF62
:1007D00015C0F4FF040EE15C03E200D0E16AE552CB
:1007E000E16EE552E7CFD9FF1200CD9ECD9CCD8AB8
:1007F000CD88CD96CD94CD82CD90CC9ECC9ACC9206
:10080000CC909F80D08EDB0EE66E0B0EE66EB6ECC3
:1008100013F0E552E5529E90F29CCD909D90F29E91
:10082000F29C1200D9CFE6FFE1CFD9FF020EE126FC
:10083000C580C5B0FED7FE0EDBCFE6FF95EC12F00B
:10084000E552DF6EFF0EDF5C04E1010EC9CFDBFF76
:10085000C69EFD0EDBCFE6FF95EC12F0E552DF6E93
:10086000C584C5B4FED7DF50146E020EE15C03E20E
:1008700000D0E16AE552E16E1450E552E7CFD9FFAE
:100880001200D9CFE6FFE1CFD9FFE6520F011C6B72
:10089000FE0EDB50F00B0809DF6E040EDF10E66E73
:1008A0001ACFE6FFBFDFE552E5520F011C6F020EC3
:1008B000E66E30DCE552FB0EDF14E66E1ACFE6FF83
:1008C000B1DFE552E5520F011C6F020EE66E22DC2D
:1008D000E552FD0EDB5023E0FE0EDB38F00BF00B93
:1008E0000809DF6E040EDF10E66E1ACFE6FF9ADF0E
:1008F000E552E5520F011C6F020EE66E0BDCE5526D
:10090000FB0EDF14E66E1ACFE6FF8CDFE552E552F0
:100910000F011C6F020EE66E8AEC00F0E552E55204
:10092000E552E7CFD9FF1200D9CFE6FFE1CFD9FFDB
:10093000E652FE0EDB50F00B08090109DF6E040ED3
:10094000DF10E66E1ACFE6FF6DDFE552E5520F01CC
:100950001C6F020EE66E8AEC00F0E552FB0EDF140F
:10096000E66E1ACFE6FF5EDFE552E5520F011C6F1F
:10097000020EE66E8AEC00F0E552FE0EDB38F00B5C
:10098000F00B08090109DF6E040EDF10E66E1ACFC6
:10099000E6FF48DFE552E5520F011C6F020EE66EDE
:1009A0008AEC00F0E552FB0EDF14E66E1ACFE6FF8C
:1009B00039DFE552E5520F011C6F020EE66E8AEC3C
:1009C00000F0E552E552E552E7CFD9FF1200320EB2
:1009D000E66EE66A9AEC00F0E552E552E66A300E01
:1009E000E66E4FDFE552E552320EE66EE66A9AECAD
:1009F00000F0E552E552E66A300EE66E42DFE5525F
:100A0000E552020EE66EE66A9AEC00F0E552E55217
:100A1000E66A300EE66E35DFE552E552020EE66E0E
:100A2000E66A9AEC00F0E552E552E66A200EE66EC0
:100A300028DFE552E552020EE66EE66A9AEC00F017
:100A4000E552E552010EE66E280EE66E1ADFE5521B
:100A5000E552020EE66EE66A9AEC00F0E552E552C7
:100A6000010EE66E080EE66E0CDFE552E552020E50
:100A7000E66EE66A9AEC00F0E552E552010EE66E8B
:100A8000E66EFFDEE552E552020EE66EE66A9AEC8D
:100A900000F0E552E552010EE66E060EE66EF1DE5E
:100AA000E552E552020EE66EE66A9AEC00F0E55277
:100AB000E552010EE66E0C0EE66EE3DEE552E552FF
:100AC000020EE66EE66A9AEC00F0E552E55212007C
:100AD000D9CFE6FFE1CFD9FF020EE126DE6ADD6A5B
:100AE000FD0EDBCFF6FFFE0EDBCFF7FF0800F55063
:100AF00021E0DECF14F0DDCF15F0D890155004E6DC
:100B0000140E145C000E155815E2FD0EDBCFF6FF37
:100B1000FE0EDBCFF7FF0800F550E66E05DFE5526D
:100B2000FD0EDB2AFE0E01E3DB2ADF2A010E01E3C4
:100B3000DB2AD6D7020EE15C02E2E16AE552E16E01
:100B4000E552E7CFD9FF1200D9CFE6FFE1CFD9FFB9
:100B5000020EE126DE6ADD6AFD0EDBCFE9FFFE0E46
:100B6000DBCFEAFFEF5020E0DECF14F0DDCF15F051
:100B7000D890155004E6140E145C000E155814E2BB
:100B8000FD0EDBCFE9FFFE0EDBCFEAFFEF50E66E96
:100B9000CBDEE552FD0EDB2AFE0E01E3DB2ADF2A67
:100BA000010E01E3DB2AD8D7020EE15C02E2E16A22
:100BB000E552E16EE552E7CFD9FF1200D9CFE6FF4B
:100BC000E1CFD9FFE652FD0EDBCF14F0FE0EDBCFF6
:100BD00015F0166A1634000E161807E6D880FA0EBD
:100BE0001454FF0E1554000E165404E2FD0EDB6A79
:100BF000FE0EDB6A300EDF6EFD0EDBCF14F0FE0E54
:100C0000DBCF15F0100E145C270E15580CE3DF2A0D
:100C1000D950FD0FE96EFF0EDA20EA6E100EEE5E7F
:100C2000270EED5AE9D70101300E6E6FDF5C02E04E
:100C3000DFCF6EF1300EDF6EFD0EDBCF14F0FE0E57
:100C4000DBCF15F0E80E145C030E15580CE3DF2A19
:100C5000D950FD0FE96EFF0EDA20EA6EE80EEE5E67
:100C6000030EED5AE9D70101300E6F6FDF5C02E031
:100C7000DFCF6FF1300EDF6EFD0EDBCF14F0FE0E16
:100C8000DBCF15F0640E145C000E15580CE3DF2A60
:100C9000D950FD0FE96EFF0EDA20EA6E640EEE5EAB
:100CA000000EED5AE9D70101300E706FDF5C02E0F3
:100CB000DFCF70F1300EDF6EFD0EDBCF14F0FE0ED5
:100CC000DBCF15F00A0E145C000E15580CE3DF2A7A
:100CD000D950FD0FE96EFF0EDA20EA6E0A0EEE5EC5
:100CE000000EED5AE9D70101300E716FDF5C02E0B2
:100CF000DFCF71F1FD0EDBCF14F0FE0EDBCF15F070
:100D0000300E1424726FFC0EDB50156A6E0F146ED9
:100D1000010E152214C0F3FF15C0F4FF00D0E552F8
:100D2000E552E7CFD9FF1200F00EE66E490EE66EEF
:100D3000020EE66EE66AE3DCE552E552E552E55264
:100D4000C2EC00F089980F01600E046F000E056F71
:100D500004CF02FF05CF03FF01011C0E5C6F010EE3
:100D60005D6F0F011E6B1E8D1E891E951E9B1E97AB
:100D70001E911E930D6B0E6B0B6B0C6B1D9FD7ECB6
:100D800000F00C0EE66E57EC01F0E552400EE66EF8
:100D90000D0EE66E030EE66EE66AB1DCE552E55234
:100DA000E552E55267EC01F001011C0E5C6F010E8B
:100DB0005D6F5CC1E6FF5DC1E6FF20EC01F0E5522E
:100DC000E552F3CF14FFF4CF15FF67EC01F00101FA
:100DD0001C0E5C6F010E5D6F18C114F019C115F087
:100DE000166A14C0E6FF15C0E6FF16C0E6FF5CC138
:100DF000E6FF5DC1E6FF07EC12F0176E050EE15E3F
:100E000017505CC1E6FF5DC1E6FF20EC01F0E55242
:100E1000E552F3CF14FFF4CF15FF01011C0E5C6FF8
:100E2000010E5D6F1AC114F01BC115F0166A14C0D3
:100E3000E6FF15C0E6FF16C0E6FF5CC1E6FF5DC138
:100E4000E6FF07EC12F0176E050EE15E17505CC16D
:100E5000E6FF5DC1E6FF20EC01F0E552E552F3CF7D
:100E600014FFF4CF15FF01011C0E5C6F010E5D6FC6
:100E700000C114F001C115F0166A14C0E6FF15C0D8
:100E8000E6FF16C0E6FF5CC1E6FF5DC1E6FF07ECCA
:100E900012F0176E050EE15E17505CC1E6FF5DC1F2
:100EA000E6FF20EC01F0E552E552F3CF14FFF4CF5A
:100EB00015FF01011C0E5C6F010E5D6F02C114F085
:100EC00003C115F0166A14C0E6FF15C0E6FF16C090
:100ED000E6FF5CC1E6FF5DC1E6FF07EC12F0176EAE
:100EE000050EE15E17505CC1E6FF5DC1E6FF20EC38
:100EF00001F0E552E552F3CF14FFF4CF15FF04C122
:100F0000E6FF05C1E6FFE7EC00F0E552E552F3CF5E
:100F100014FFF4CF15FFC69A0F014E0E1A6F800E04
:100F2000E66E080EE66ED2EC13F0E552E552180EAE
:100F3000C86EC750040B01E0010E146E1F0EC514DD
:100F4000141001E0F6D7C580C5B0FED7C9CF1BFF8E
:100F50001ACFE6FF95EC12F0E5520F011C6FFF0E61
:100F60001C5D03E1C9CF1BFFC69E122B000E13238D
:100F70001C5105E0640E125D000E1359E9E3640E86
:100F8000125D000E135920E212CFE6FF13CFE6FFE9
:100F90001A51E66EE66AFE0E146E210E156E166A82
:100FA00014C0E6FF15C0E6FF16C0E6FFFE0EE66EB3
:100FB000E668B9EC11F0176E090EE15E1750F3CF39
:100FC00014FFF4CF15FF22D012CFE6FF13CFE6FFB8
:100FD0001C51E66EE66A1A51E66EE66AC40E146E9D
:100FE000210E156E166A14C0E6FF15C0E6FF16C086
:100FF000E6FFFE0EE66EE668B9EC11F0176E0B0E1A
:10100000E15E1750F3CF14FFF4CF15FF67EC01F04A
:10101000ADEC03F001011C0E5C6F010E5D6F0AC1A7
:1010200014F00BC115F0166A14C0E6FF15C0E6FFF8
:1010300016C0E6FF5CC1E6FF5DC1E6FF07EC12F0FB
:10104000176E050EE15E17505CC1E6FF5DC1E6FF5D
:1010500020EC01F0E552E552F3CF14FFF4CF15FF79
:1010600067EC01F0B4DC0F011C51E66EE66AA70ED6
:10107000146E210E156E166A14C0E6FF15C0E6FF49
:1010800016C0E6FFFE0EE66EE668B9EC11F0176ECC
:10109000070EE15E1750F3CF14FFF4CF15FF0F01D9
:1010A0001C6B010EE66EE66E41EC04F0E552E55273
:1010B000010EE66E020EE66E41EC04F0E552E552DA
:1010C000010E0F01126F136B67EC01F0010EE66E5B
:1010D000E66ABBEC03F0E552E552F3CF16FFF4CF1E
:1010E00017FF16CFE6FF17CFE6FF12CFE6FF13CFAD
:1010F000E6FF900E146E210E156E166A14C0E6FF00
:1011000015C0E6FF16C0E6FFFE0EE66EE668B9EC17
:1011100011F0176E090EE15E1750F3CF14FFF4CFF4
:1011200015FF0F01460E1A6F121D1B6F1BCFE6FF36
:101130001ACFE6FF12EC04F0E552E5520F011C6FE6
:101140001C51E66EE66A1B51E66EE66A6F0E146E7F
:10115000210E156E166A14C0E6FF15C0E6FF16C014
:10116000E6FFFE0EE66EE668B9EC11F0176E090EAA
:10117000E15E1750F3CF14FFF4CF15FF0F014E0EB1
:101180001A6F25DC880EE66E130EE66EE66AE66AD6
:101190007FEC03F0E552E552E552E552010EE66EB2
:1011A000E66E41EC04F0E552E552010EE66E020EE9
:1011B000E66E41EC04F0E552E55201011C0E5C6F55
:1011C000010E5D6F06C114F007C115F0166A14C058
:1011D000E6FF15C0E6FF16C0E6FF5CC1E6FF5DC195
:1011E000E6FF07EC12F0176E050EE15E17505CC1CA
:1011F000E6FF5DC1E6FFA8DCE552E552010EE66EB2
:10120000C00EE66E41EC04F0E552E5520CC1E6FF7B
:101210000DC1E6FF5DDCE552E552010EE66E940E6F
:10122000E66E41EC04F0E552E55201011C0E5C6FE4
:10123000010E5D6F0EC114F00FC115F0166A14C0D7
:10124000E6FF15C0E6FF16C0E6FF5CC1E6FF5DC124
:10125000E6FF07EC12F0176E050EE15E17505CC159
:10126000E6FF5DC1E6FF70DCE552E552010EE66E79
:10127000D40EE66E41EC04F0E552E55201011C0E7D
:101280005C6F010E5D6F16CFE6FF17CFE6FF16CF3E
:10129000E6FF17CFE6FF5A0E146E210E156E166A82
:1012A00014C0E6FF15C0E6FF16C0E6FF5CC1E6FF0E
:1012B0005DC1E6FF14EC11F0176E090EE15E1750E8
:1012C000F3CF14FFF4CF15FF5CC1E6FF5DC1E6FF6D
:1012D0003BDCE552E552900EE66ED00EE66E030E54
:1012E000E66EE66A7FEC03F0E552E552E552E55220
:1012F0000F01122B000E1323FF0E1215126F136B2A
:1013000067EC01F0E3D61200C0EC0EF0FB0EDBCF71
:10131000F3FFDB06F35000090AE00EEC0FF0FA0EC3
:1013200079EC0FF0F3E1151CF1E1010E01D0000E94
:10133000EFEF0EF0C0EC0EF03B0EE12402E3E168AB
:10134000E652E16E010EDB6A020EDB6AF90EDBCFBC
:10135000F6FFFA0EDBCFF7FFFB0EDBCFF8FF08003E
:10136000F550DF6EDF5002E113EF0EF0250EDF5C6B
:1013700002E006EF0EF0030EDB6A040EDB6A050ED8
:10138000DB6A060EDB6A070EDB6A28EC0EF02D0E18
:10139000DF5C0CE02B0EDF5C09E0200EDF5C06E07A
:1013A000230EDF5C03E0300EDF5C1AE1DF50300A11
:1013B00014E0130A0FE0030A0AE00B0A05E0060A2C
:1013C000E4E1030EDB80E1D7030EDB82DED7030E00
:1013D000DB84DBD7030EDB86D8D7030EDB88D5D7BB
:1013E0002A0EDF5C1BE124EC0EF072EC0EF010E034
:1013F000030EDB8006680768130EDBCF0DF0140EBA
:10140000DBCF0EF046EC13F0040E04C0DBFF03D07C
:10141000130E5BEC0EF028EC0EF00BD0090EDB6A1D
:10142000C9EC0EF003E03DEC0FF0FAD7090E5BECCF
:101430000EF0030EDBB0DB982E0EDF5C1BE128EC18
:101440000EF02A0EDF5C0BE124EC0EF072EC0EF0D5
:1014500003E1130EADEC0EF028EC0EF00BD0090EEC
:10146000DB6AC9EC0EF003E03DEC0FF0FAD7090E91
:10147000ADEC0EF0680EDF5C07E128EC0EF0680EB4
:10148000DF5C1DE1030E18D0740EDF5C17E07A0EEE
:10149000DF5C14E0480EDF5C06E0540EDF5C03E026
:1014A0005A0EDF5C02E1020E07D06C0EDF5C03E037
:1014B0006A0EDF5C04E1010E00EC0FF0C9DBDF50C7
:1014C0006E0A01E17FD31E0A01E192D1200A01E1F7
:1014D0008FD13F0A01E149D11A0A01E146D10D0A33
:1014E00001E143D1200A01E140D13A0A01E13DD1B5
:1014F000200A01E13AD1260A01E135D10D0A01E1C4
:1015000032D11A0A01E1D9D0200A4AE0300A1FE09C
:10151000460A0EE0250A01E083D3D950F90FE96E9F
:10152000FF0EDA20EA6E010EEE5E000EEE5AEE5A63
:101530000EEC0FF0250EE66E95DB03E1151C01E1C4
:1015400069D30AEC0FF001E26BD3DB2A69D3080EF2
:10155000DB6A040EDB50010806E2040EDB04D2EC69
:101560000EF0DB508BDB080EDB5009E0030EDB5086
:10157000010B05E172DB01E04DD3080EDB6A64DB91
:10158000EFCFDFFF82EC0FF003E1151C01E142D346
:101590000AEC0FF001E3DB2A60DB01E141D33AD32F
:1015A000070EDB5002080FE14EEC0FF0030E15ECB6
:1015B0000FF00E0EEECFDBFF0F0EEECFDBFF100EA7
:1015C000EECFDBFF20D0F70EDBCF17F0F80EDBCF2E
:1015D00018F0020E175E000E185AF70E17C0DBFF48
:1015E000F80E18C0DBFF17C0E9FF18C0EAFF05ECD2
:1015F0000FF0166A0E0E14C0DBFF0F0E15C0DBFFD6
:10160000100E16C0DBFF0E0EDBCFE6FF0F0EDBCF9A
:10161000E6FF100EDBCFE6FF2EEC12F0E552E552AE
:10162000E552130E05C0DBFF140E06C0DBFF060EED
:10163000DB5005E0130E49EC0FF001E26ADB6DECC4
:101640000FF002E2130E37DB30EC0FF006E0040E71
:1016500049EC0FF002E2050E2EDB030EDBB005D0E5
:10166000FCDA01E0D7D2080EDB6A090EDB6A0E0E47
:10167000DBCFF6FF0F0EDBCFF7FF100EDBCFF8FF4F
:101680000800F550DF6EDF5014E073EC0FF011E24C
:1016900082EC0FF003E1151C01E1BCD2BBDB01E3DE
:1016A000DB2A090EDB2AD9500E0FE96E000ECBDBC8
:1016B000E7D7D3DA01E1B4D2ADD2C6DA110EEECF5C
:1016C000DBFF120EEDCFDBFF110EDBCFE6FF120EBC
:1016D000DBCFE6FF20EC12F0E552E552130EF3CF1C
:1016E000DBFF140EF4CFDBFF060EDB5004E0130E1D
:1016F000D0DB01E20EDB6DEC0FF002E2130EDBDA61
:10170000AFDB05E0040EC5DB02E2050ED4DA030E02
:10171000DBB005D0A2DA01E07DD2080EDB6A090E4B
:10172000DB6A110EDBCFE9FF120EDBCFEAFFEFCF52
:10173000DFFFDF5014E0D7DB12E2E4DB03E1151C2E
:1017400001E168D267DB01E3DB2A090EDB2A110E17
:10175000DB2ADBCFE9FF120EE8E3DB2AE6D77DDAEE
:1017600001E15ED257D2030EDB8E070EDB0410E1DF
:1017700095DB040E5ADB0A0EEECFDBFF0B0EEECF2D
:10178000DBFF0C0EEECFDBFF0D0EEECFDBFF6CD0E0
:10179000070EDB5003082CE1030EDBAE0DD0B2DAEE
:1017A000020E76DAEFCF14F0156A166A176A14AED5
:1017B00039D01568166835D0F70EDBCF15F0F80E66
:1017C000DBCF16F0020E155E000E165AF70E15C08E
:1017D000DBFFF80E16C0DBFF15C0E9FF16C0EAFFFD
:1017E000EFCF14F00A0E14C0DBFF0B0EDB6A38D00B
:1017F000070EDB50020809E1030EDBAE04D059DB13
:1018000016AE10D00ED055DB0DD0030EDBAE12D0CD
:1018100079DA020E3DDAF9DA166A176A15AE02D0E5
:1018200016681768E2DA0C0E16C0DBFF0D0E17C043
:10183000DBFF1AD0F70EDBCF16F0F80EDBCF17F078
:10184000020E165E000E175AF70E16C0DBFFF80EDA
:1018500017C0DBFF16C0E9FF17C0EAFFD6DAC5DA0A
:101860000C0EDB6A0D0EDB6A060EDB5005E1010E85
:10187000F36E050EF3CFDBFF150EDB6A160EDB6A87
:10188000D950370F146E000EDA20156E390E14C0C1
:10189000DBFF3A0E15C0DBFF380EDB6A080EDB6A91
:1018A0000A0EAEDADF50780A12E0200A10E0280AA9
:1018B0000CE0200A0AE03F0A06E00D0A02E0200AD6
:1018C00008E1020E05D0080E03D0080EDF26100E28
:1018D00097DA030EDBBE02D0DB92DB94DB50800B89
:1018E00024E08ADAD890030EEB50000A08E6000ED6
:1018F000EE5C000EEE58000EEE58000EEE5815E2AB
:1019000013DA0B680C680D680E680EEC13F00A0E03
:1019100000C0DBFF0B0E01C0DBFF0C0E02C0DBFFC3
:101920000D0E03C0DBFF2D0E08D0030EDBA202D08C
:101930002B0E03D0DBA408D0200EF36E170EF3CFCE
:10194000DBFF150EDB2A02D0170EDB6A050EDB501B
:1019500003E1B7D901E189D0A80E146E280E156EE7
:10196000000E166E070EDBCF17F0186A196A1A6A96
:1019700017C00BF018C00CF019C00DF01AC00EF013
:10198000D3D973EC13F014500024F36E15500120DA
:10199000F46E16500220F86EF4CFF7FFF3CFF6FF87
:1019A0000800090EF5CFDBFF580EDF5C0FE1610E7A
:1019B000F36E090E7BD90AE3200E146E090EDBCFFD
:1019C000E7FF1450E75E090EE7CFDBFF070EDBCF22
:1019D00014F0156A166A176A0FDA14C00BF015C0F6
:1019E0000CF016C00DF017C00EF0EECF04F0EECFE5
:1019F00005F0EECF06F0EFCF07F073EC13F007C061
:101A0000EDFF06C0EDFF05C0EDFF04C0EFFF390E8E
:101A1000DBCFE9FFDB063A0EDBCFEAFF01E2DB06B4
:101A2000090EDBCFEFFF150EDB2A4BD995E1030E34
:101A3000DBA61DD06F0EDF5C06E1C1D918E3150EE1
:101A4000DB285BDA14D0780EDF5C09E0580EDF5C2F
:101A500006E0620EDF5C03E0420EDF5C08E1020E8E
:101A6000F36E160EF3CFDBFF02D0150EDB6A030E0A
:101A7000DB50100B0EE0040EDBCF14F0050EDB5034
:101A8000D880145406E2060EDB5003E1040EDB504E
:101A900034DA95D90AE2050EDBCFE7FF150EDB50ED
:101AA000E75E050EE7CFDBFF02D0050EDB6A040E12
:101AB000DBCF14F0160E45D9D880145414E2160E5C
:101AC000DBCFE6FF150EDBCFE6FF040EDBCFE6FF34
:101AD000050EDB50E552E75CE552D880E754E5524D
:101AE000D880E7545FD9030EDB50010B0BE1080EE1
:101AF000DB5008E0B2D801E08DD0080EDB50BED834
:101B0000080EDB6A170EDB5007E088D9170EF1D9F3
:101B100003E1151C01E17ED0160EDB5016E07ED9E4
:101B2000300EE66E9FD802E1151C74E077D9DFCF46
:101B3000E6FF53EC12F0E552E552E552F4CF15F012
:101B40000001F31C02E1151C65E0050EDBCF14F06B
:101B5000160EDB50D880145409E2050EDBCFE7FFE8
:101B6000160EDB50E75E050EE7CFDBFF300EE66EAC
:101B7000050ECBD94FE1390EDB2ADBCFE9FF3A0E58
:101B800001E3DB2ADBCFEAFF090EEFCFDBFFDB50FF
:101B90000EE044D9090EADD902E1151C3BE0390E27
:101BA000DB2ADBCFE9FF3A0EEDE3DB2AEBD755D892
:101BB00031E1160EDBCFE6FF080EC3D8E552E7246D
:101BC0005DD82ED0070EDB50030A1CE0010A14E09A
:101BD000030A07E07BD9DBCFEEFF020EDBCFEDFF80
:101BE0001FD0F5D8196A17AE02D0186819682CD81A
:101BF000BCD819C0EEFF14D0EAD817BE186824D894
:101C0000B4D80ED063D9DBCFEFFF0AD07BD905E182
:101C1000151C03E1F368F46810D0FCD801E3DB2A5B
:101C200079D9AFEF09F0010EDBCF14F0020EDBCF54
:101C300015F014C0F3FF15C0F4FF3B0EE15C02E2A7
:101C4000E16AE552E16ECBD029D9020E15EF0FF013
:101C500061D90800F550DF6E1200200EE66E080E06
:101C600085EF0FF053EC12F0E552E552E552F3CF59
:101C700014F0F4CF15F00001F31C1200146E156A75
:101C8000D950010F4DD91450EE261550ED221200F7
:101C9000185E000E195AF70E18C0DBFFF80E19C0B7
:101CA000DBFF18C0E9FF19C0EAFF1200DBCFF4FF29
:101CB000F350F45C1200DB50E76E040EE7CFDBFF5D
:101CC00012000A0EDBCF14F00B0EDBCF15F00C0E5A
:101CD000DBCF16F00D0EDBCF17F0145015101610D9
:101CE00017101200130EEECFDBFF140EEDCFDBFF4B
:101CF000130EDBCF14F0140EDBCF15F00001800EB5
:101D000015141200F70EDBCF18F0F80EDBCF19F028
:101D10001200050EDB50E66ED950130F01D9E552C3
:101D2000E750EE6EED6A12000A0EDBCF04F00B0EE8
:101D3000DBCF05F00C0EDBCF06F00D0EDBCF07F08E
:101D40001200DBCFE6FF150EDBCFE6FF050EDB5002
:101D5000E552E724E552E7241200DB50CED8010E0D
:101D6000F36E060EF3CFDBFF1200EE50EFCFEAFF6B
:101D7000E96E16C0EEFF17C0EEFF18C0EEFF1200AE
:101D8000D9CFE6FFDACFE6FFE1CFD9FFE2CFDAFF26
:101D90001200DFCFE6FFE66A02EC14F0E552E552EE
:101DA000F3501200E76E080EE7CFDBFF1200EECF14
:101DB00014F0EECF15F0EFCF16F0176A1200050EF3
:101DC000DBCF14F0150EDB50D88014541200010E36
:101DD000DBCF16F0020EDBCF17F0186A1200E552C7
:101DE000E5CFDAFFE7CFD9FF12000A0E14C0DBFF00
:101DF0000B0E15C0DBFF1200D9500A0F90EF0FF049
:101E0000F36E070EF3CFDBFF1200EECF14F0EFCF2F
:101E100015F01200010EDB2A020E1200FC0EDBCFC1
:101E2000E6FFFD0EDBCFE6FF1200145E000E155A32
:101E3000F70E14C0DBFFF80E15C0DBFF14C0E9FF7E
:101E400015C0EAFF1200DA20EA6EEF2AEECFF6FFA5
:101E5000000EEF22EECFF7FFEF22EECFF8FF1200D9
:101E6000040EDBCFE6FF130EDB50E552E75C9ADF92
:101E7000DB5004DF060EDB501200090EDB500A0DAA
:101E8000F350DF24D00FE76E090EE7CFDBFF28EF1A
:101E90000EF0DB50F36E050E56EF0EF0F70EDBCFB3
:101EA00014F0F80EDBCF15F01200DFCFE6FF32EFB3
:101EB0000EF028DF030EECDED7EF0EF084EC09F015
:101EC000E552E552E552E55200091200BDDEEE5042
:101ED000EFCFEAFFE96E010E1200130EDB50F36E36
:101EE000040E56EF0EF0040EDB50F36E090E56EFA3
:101EF0000EF0DBCFE6FF32EF0EF0E76E050EE7CF18
:101F0000DBFF12008BDF55EF0FF0DBCFE6FF86DF44
:101F10005EEF0FF0D950F90FE96EFF0E23EF0FF0CF
:101F2000E96E000EDA20EA6E1200D9CFE6FFDACFB2
:101F3000E6FFFA0EE3CFD9FFFB0EE3CFDAFFFD0E8B
:101F4000E35209E72D0EDE6EFC0EE31EE32AFD0EC2
:101F5000D8B4E306E31EE652E652E652FD0EE12453
:101F6000E76EFF0EE220E46EE652F70EE3CFE6FFE7
:101F7000F70EE3CFE6FF05EC10F0F90EE124E96E71
:101F8000FF0EE220EA6EF5EC0FF00AE1F2EC0FF042
:101F900009E1F5EC0FF008E1F2EC0FF007E108D0F1
:101FA00000EC10F0FBEC0FF000EC10F0FBEC0FF08D
:101FB00000EC10F0DE6AF90EE126FF0EE222FF0EC1
:101FC000E3CFDAFFE552FF0EE3CFD9FFE552FC0E77
:101FD000E124E96EFF0EE220EA6EEECFF3FFEFCFD1
:101FE000F4FF1200EF380F0B1200EF500F0B02E15D
:101FF000EE52D8841200EF380F0B300FDE6E120055
:10200000EE500F0B300FDE6E1200FC0EE3CFE9FF37
:10201000FD0EE3CFEAFF100EE66EEE6AEE6AEF6A9F
:10202000D890FD0EE336FE0EE336ED36ED36EF3694
:10203000FF0EE30609E026EC10F0EE5226EC10F05D
:10204000EE5226EC10F0EDD7E56E1200030EEF24F1
:10205000E8B6EF6E300EEF24E8BEEF6E000C3138BC
:102060004632364B3232203130204D687A204F7361
:10207000632E2051756172747A200D00506F727456
:1020800020636F6D6D2031393230302062647320EF
:102090006F75766572740D00496E6974204932431C
:1020A000200D00496E6974204C4344203420782070
:1020B00032302063617200636C65617220736372F9
:1020C00065656E204C4344200D00496E69742041C3
:1020D0004443200D00313233343536373839302D12
:1020E000414243444546474849004A4B4C4D4E4FB8
:1020F000505152535455565758595A2D2F2A002093
:1021000020202020202020202020202020202020CF
:10211000202020003039200D003130200D003131D9
:10212000200D0031384632366B32325F4C43445F0B
:102130004932435F48617264775F6D6173746572A1
:102140002E630D0056657273696F6E203A2030352C
:102150002F30352F313320610D004D657375726559
:10216000204144433D25303464202530335800203D
:102170002020253364202D3E2050434640203078D7
:10218000343620205374617475733D253364200008
:10219000696E646963653D253033642020414443A2
:1021A000303D2530356400417072657320496E6999
:1021B00074204C4344202C207374617475733D2546
:1021C00033642000504220616472657373616765F7
:1021D00020253032582C20496E6974204932432022
:1021E000494E636F727265637465205374617475D0
:1021F000733D25336420206A3D2535640D00496E0A
:102200006974205043463835373420636F727265E5
:1022100063746520416472657373653D253032587F
:10222000206A3D2533640D00D9CFE6FFDACFE6FF03
:10223000E1CFD9FFE2CFDAFFE652E652E652E652AC
:10224000D950F90F146EFF0EDA20156E020E14C06D
:10225000DBFF030E15C0DBFF020EDBCFE6FF030E34
:10226000DBCFE6FFF90EDBCFE6FFFA0EDBCFE6FFB2
:10227000FB0EDBCFE6FFD950FC0FE66EFF0EDA2037
:10228000E66E9AEC09F0146E070EE15C02E2E16A78
:10229000E552E16E1450F3CFDEFFF4CFDDFFFC0E0C
:1022A000DBCFE9FFFD0EDBCFEAFFEF6ADECF14F0F4
:1022B000DDCF15F014C0F3FF15C0F4FF040EE15C90
:1022C00002E2E16AE552E16EE552E5CFDAFFE7CFDF
:1022D000D9FF12000E0EF66E000EF76E000EF86EAD
:1022E0000F010900F5502D6F0900F5502E6F03E125
:1022F0002D6701D03DD00900F550286F0900F55039
:10230000296F0900F5502A6F09000900F550E96EA0
:102310000900F550EA6E090009000900F5502B6F1D
:102320000900F5502C6F09000900F6CF2FFFF7CFF9
:1023300030FFF8CF31FF28CFF6FF29CFF7FF2ACFA4
:10234000F8FF0F012B5302E12C5307E00900F55071
:10235000EE6E2B07F8E22C07F9D72FCFF6FF30CF20
:10236000F7FF31CFF8FF0F012D07000E2E5BBFD70F
:102370001200D9CFE6FFDACFE6FFE1CFD9FFE2CFF7
:10238000DAFFE652E652E652E652D950F90F146EE1
:10239000FF0EDA20156E14C0DEFFDD6EDECFE6FF25
:1023A000DDCFE6FFF90EDBCFE6FFFA0EDBCFE6FF6F
:1023B000FB0EDBCFE6FFFC0EDBCFE6FFFD0EDBCF37
:1023C000E6FF9AEC09F0146E070EE15C02E2E16AA6
:1023D000E552E16E1450020EF3CFDBFF030EF4CF93
:1023E000DBFF020EDBCF14F0030EDBCF15F014C0C1
:1023F000F3FF15C0F4FF040EE15C02E2E16AE5526E
:10240000E16EE552E5CFDAFFE7CFD9FF1200FB0E10
:10241000E3CFF6FFFC0EE3CFF7FFFD0EE3CFF8FFAF
:10242000FE0EE3CFE9FFFF0EE3CFEAFFE9CFF3FFB4
:10243000EACFF4FF0900F5CFEFFFEE66FBD71200FD
:10244000FE0EE3CFE9FFFF0EE3CFEAFFF36AF46A83
:10245000EE5203E0F34AF42AFBD71200FF0EE3CF5B
:10246000F8FFE552FF0EE3CFF7FFE552FF0EE3CF93
:10247000F6FFE552E66AE66AE66A0900F55209E007
:10248000FD0EE32A05E1FE0EE32A02E1FF0EE32A38
:10249000F4D7FD0EE3CF05F0FE0EE3CF06F0FF0EFE
:1024A000E3CF07F01200D9CFE6FFDACFE6FFE1CFA6
:1024B000D9FFE2CFDAFFFB0EDBCF14F0FC0EDBCF4F
:1024C00015F00001800E15141AE1FB0EDBCFE9FFB9
:1024D000FC0EDBCFEAFFEECFF3FFEDCFF4FFEE2AE9
:1024E000000EEF22F3CFE9FFF4CFEAFFFD0EDBCFC2
:1024F000EFFFEF50156AF36E15C0F4FF10D0FB0E1E
:10250000DB50FE0806E1FD0EDBCFE6FF32EC14F0F7
:1025100005D0FD0EDBCFE6FF03EC00F0E552E552FF
:10252000E5CFDAFFE7CFD9FF1200D9CFE6FFDACF48
:10253000E6FFE1CFD9FFE2CFDAFFFD0EDB50C96E37
:10254000C6AE02D0FF0E2BD00F0EC61408080FE047
:102550000F0EC6140B080BE0C6889EA6FED7C75008
:10256000040B03E1C750010B17E0000E18D00F0E4B
:10257000C614080804E00F0EC6140B0810E1C7B01B
:10258000FED7C750040B01E0010E146E1F0EC514D8
:102590001410F7E1C5AC02D0FE0E01D0000EE552DA
:1025A000E5CFDAFFE7CFD9FF1200D9CFE6FFDACFC8
:1025B000E6FFE1CFD9FFE2CFDAFFAC6AAB6AFD0EEE
:1025C000DBB0AC88DBA202D0AC8CAB8CDBB4AC8EC5
:1025D000DBA602D0AB8801D0AB8ADBB8AC84DBBA17
:1025E000AB86DBAC02D09D8A01D09D9ADBAE02D0D7
:1025F0009D8801D09D98FB0EDB50AF6EFC0EDBCFAB
:1026000015F015C014F0156A1450B06EAC8AAB8E7C
:10261000E552E5CFDAFFE7CFD9FF120004500B02F5
:10262000F3CF00F0F4CF01F00C02F3500126000EBE
:10263000F420026E04500D02F3500226000EF42026
:10264000036E04500E02F350032605500B02F350A4
:102650000126F4500222000E032205500C02F35012
:102660000226F450032205500D02F35003260650B3
:102670000B02F3500226F450032206500C02F350D2
:10268000032607500B02F3500326120007C013F075
:1026900006C012F006500D02F4CF05F0F3CF04F09F
:1026A00007500E02F4CF07F0F3CF06F00D02F350FF
:1026B0000526F4500622E86A072212500E02F35053
:1026C0000526F4500622E86A07220EAE6CEF13F0DE
:1026D0001250065E1350075A13AE000C0D50065EE2
:1026E0000E50075A000C036A026A016A006A200E43
:1026F000E76ED890043605360636073600360136C2
:10270000023603360B50005C0C5001580D50025835
:102710000E50035809E30B50005E0C50015A0D5047
:10272000025A0E50035A042AE72EE4D71200D9CFDA
:10273000E6FFDACFE6FFE1CFD9FFE2CFDAFFE652DC
:10274000F20E0F013217ABAC03D03291ABB0328135
:10275000ABB43285ABB23287AE50DF6EDF50E5529C
:10276000E552E5CFDAFFE7CFD9FF1200D9CFE6FF78
:10277000DACFE6FFE1CFD9FFE2CFDAFFE652E65249
:10278000FC0EDBCFDEFFDBCFDDFF010EDB50CF6EBB
:10279000DF50CE6EE552E552E552E5CFDAFFE7CFE6
:1027A000D9FF1200D9CFE6FFDACFE6FFE1CFD9FF9C
:1027B000E2CFDAFF3F0EC716C66AC56AFD0EDB50D0
:1027C000C612FC0EDB50C712C68AE552E5CFDAFF0F
:1027D000E7CFD9FF1200D9CFE6FFDACFE6FFE1CF8E
:1027E000D9FFE2CFDAFFACAC04D0AC900F0132B32A
:1027F000AC80FD0EDB50AD6EE552E5CFDAFFE7CFE2
:10280000D9FF1200F36AF46AFF0EE124E96EFF0EAD
:10281000E220EA6EED6607D02F0EEF6404D03A0E88
:10282000EF6001D0F32A1200380EF36E00EE00F0D4
:102830000F0E01D81200EA6002D0EE6AFCD7F35006
:10284000E9601200EE6AFCD71EEE00F02EEE00F0FA
:10285000F86A0A9C6AEC11F064EC14F094EC06F04F
:10286000FBD71200FF0EE350ACBA04D0AF6AAB8EB8
:10287000AC8A949CACA2FED7AD6EF36EF46A1200E3
:10288000FF0EE350E84E1200000000D000D000D050
:10289000E82EFAD71200C450176E166AC3501610ED
:1028A000F36E17C0F4FF120030313233343536374F
:1028B000383961626364656600FFC250020B01E053
:1028C000010E1200C282120012005E207C209820AD
:1028D000A320B720CA20D520EA20FF2014211921E7
:1028E0001E212321442150524F4A45543A20313869
:1028F0004632364B32325F4C43445F4932432E6D91
:1029000063700000000000000000000000000000F4
:1029100000000000000000000000000000000000B7
:102920000000000000001C013132333435363738E6
:102930003930313233343500303030303000FFFF41
:10294000FFFFFFFFFFFFFFFFFFFFFFFFFFFFFFFF97
:10295000FFFFFFFFFFFFFFFFFFFFFFFFFFFFFFFF87
:10296000FFFFFFFFFFFFFFFFFFFFFFFFFFFFFFFF77
:10297000FFFFFFFFFFFFFFFFFFFFFFFFFFFFFFFF67
:0200000400F00A
:100000002031384632364B3232203130204D687A3A
:100010002073616E7320504C4C202020200D000076
:1000200020506F727420436F6D203139323030624E
:100030006473204F7576657274202020200D0000B7
:1000400020496E6974204C43442034783230636117
:10005000722049324320202020202020200D000043
:100060002020202020202020202020202020202090
:10007000202020202020202020202020200D0000D3
:100080002020202020202020202020202020202070
:10009000202020202020202020202020200D0000B3
:1000A0002020202020202020202020202020202050
:1000B000202020202020202020202020200D000093
:1000C0002020202020202020202020202020202030
:1000D000202020202020202020202020200D000073
:1000E0002020202020202020202020202020202010
:1000F000202020202020202020202020200D000053
:1001000020202020202020202020202020202020EF
:10011000202020202020202020202020200D000032
:1001200020202020202020202020202020202020CF
:10013000202020202020202020202020200D000012
:1001400020202020202020202020202020202020AF
:10015000202020202020202020202020200D0000F2
:10016000202020202020202020202020202020208F
:10017000202020202020202020202020200D0000D2
:10018000202020202020202020202020202020206F
:10019000202020202020202020202020200D0000B2
:1001A000202020202020202020202020202020204F
:1001B000202020202020202020202020200D000092
:1001C000202020202020202020202020202020202F
:1001D000202020202020202020202020200D000072
:1001E0002030352F30352F3133206120207061755C
:1001F0006C666A756A6F200D000101010101010141
:1002000076657273696F6E30352F30352F3133203C
:1002100061200000313020202020202020202020BC
:10022000202020200000000032302020202020202C
:10023000202020202020202000000000333020201B
:10024000202020202020202020202020000000002E
:10025000343020202020202020202020202020207A
:1002600000000000353020202020202020202020E9
:1002700020202020000000003630202020202020D8
:1002800020202020202020200000000037302020C7
:1002900020202020202020202020202000000000DE
:1002A0003830202020202020202020202020202026
:1002B0000000000039302020202020202020202095
:1002C000202020200000000041302020202020207D
:1002D000202020202020202000000000423020206C
:1002E000202020202020202020202020000000008E
:1002F00043302020202020202020202020202020CB
:100300000000000044302020202020202020202039
:100310002020202000000000453020202020202028
:100320002020202020202020000000004630202017
:10033000202020202020202020202020000000003D
:10034000FFFFFFFFFFFFFFFFFFFFFFFFFFFFFFFFBD
:10035000FFFFFFFFFFFFFFFFFFFFFFFFFFFFFFFFAD
:10036000FFFFFFFFFFFFFFFFFFFFFFFFFFFFFFFF9D
:10037000FFFFFFFFFFFFFFFFFFFFFFFFFFFFFFFF8D
:10038000FFFFFFFFFFFFFFFFFFFFFFFFFFFFFFFF7D
:10039000FFFFFFFFFFFFFFFFFFFFFFFFFFFFFFFF6D
:1003A000FFFFFFFFFFFFFFFFFFFFFFFFFFFFFFFF5D
:1003B000FFFFFFFFFFFFFFFFFFFFFFFFFFFFFFFF4D
:1003C000FFFFFFFFFFFFFFFFFFFFFFFFFFFFFFFF3D
:1003D000FFFFFFFFFFFFFFFFFFFFFFFFFFFFFFFF2D
:1003E000FFFFFFFFFFFFFFFFFFFFFFFFFFFFFFFF1D
:1003F000FFFFFFFFFFFFFFFFFFFFFFFFFFFFFFFF0D
:020000040030CA
:0E0000000022193C009D84000FC00FE00F404D
:020000040020DA
:08000000FFFFFFFFFFFFFFFF00
:00000001FF
